:03000000020027D4
:04000B00120170323C
:10002300120205327590FF75B0CB53D0E775810F7F
:10003300C2AFC28CC28EC23F754C087589217598B8
:10004300F0538700758C00758A00758DFD758BFDE7
:10005300D28E75B802D2AFD2A91200C512018BD2CB
:10006300ACD29D30380920B706D23AC239C2382003
:100073003C05103E1980EC75483C754722203B0A2D
:10008300D547FAD548F7C23CD29DC23B80D5E5415E
:10009300B405051200A380CBB406031200A880C3E5
:1000A30012012AE4221200E8D238C3E54C1370018E
:1000B30033F54C203903754C08854C4BD239D28C1F
:1000C300E422C2B5C2B4C2B37A027928D2B400D250
:1000D300B500C2B500C2B400D2B500C2B500D9F8AC
:1000E300DAE8D29022C2AFC2B390027378387A04AE
:1000F300D2B400D2B500C2B500E6C3942093A237B0
:1001030092E079083392B400D2B500C2B500D9F4B5
:1001130008DAE6E654C079063392B400D2B500C2D9
:10012300B500D9F4D2AF22C2A9D2B2120157E4A2C8
:10013300B733F5993099FDC299F5993099FDC29974
:1001430012014DC2B2C23AD2A922754A01754910B1
:1001530012016122754A0175499A12016122D5493A
:10016300FDD54AFA22E590C4540FF5402230390FE9
:10017300D54B0BB237B29011E8854C4BD23622C225
:100183008CC237D29011E822854C4BC236D239D279
:100193008CD2D37A007C1A9001E87B047838A90AC0
:1001A300E993F60809DBF9C2D310360280FBD2D3F8
:1001B3000ADCE431682430B439030201C440022468
:1001C3000718F6C2D37548FF7547FF00000000000B
:1001D300000000000000D547F2D548EF11C5C28CDE
:1001E300C239D290222020202053454C462074450A
:1001F3005374203031323334353637383920416443
:10020300642020980122C0E0C0D0D2D3D23B85998C
:1002130045309A1E3168E54575F010846003B5409A
:100223004885F041C29DD23DD23CE4F544F54302FA
:10023300026CE545303D13F546C23D7406B54105F4
:10024300793802026C793002026C0543E543B54606
:1002530010E544B545041546D23ED29DC23C020288
:100263006CE545F76544F54409D0D0D0E0C2982247
:1002730000004400000000409CF000000402000065
:10028300FC60DAF266B6BEE0FEF60000000000CACB
:1002930000EEFE9CFC9E8EBC6E60F8001C0000FC11
:1002A300CE0000B6007C00000000009D00F00010AE
:1002B30004FA3E1A7ADE8EF62E40780060002A3A5F
:0B02C300CE000AB61E380000007600D6
:00000001FF
